:020000040000FA
:0600000014D0D9D013D08A
:02000800FFD027
:06000A0082BEFED70400D7
:0600100082AEFED71200D3
:02001800FFD017
:06002A00EAD0949C900E48
:10003000AB6E260EAC6EAB98030ED56ED76AD66A41
:10004000E4DFD58EE2DFD59ED6CF03F0D732033280
:10005000D8A0030603C0AFFFAB88AE50AE50A3D804
:100060000F0AE9E100EE08F0006A016A9CD80F0A65
:10007000F6E00450040A0AE00450050A01E193D8AE
:1000800004500026EE6E014ED6D7F0D70052D3E1D1
:100090000A50F66EA96E0B50F76EAA6E0CC0F8FFF0
:1000A00000EE0DF00950016ED8B4FF0008500708AB
:1000B000C2E3FA6AFB6A0844F92607D00CD013D0D1
:1000C00022D02CD036D007D040D00B0E0A6E000EB6
:1000D0000B6E040E45D00900F5CFEEFF012EFBD7C5
:1000E0000950050F3DD0F80EF616080EEECFF5FFBD
:1000F0000D00E82EFBD70A00840EA66E5CD809001E
:10010000012EF1D72CD0940EA66E55D8400EF626AF
:10011000E86AF722F822012EF6D721D0A66AA68037
:10012000A8CFEEFFA94AAA2A012EF8D70950050F39
:1001300017D0EECFA8FF040EA66E3DD8A6B2FED70C
:10014000A94AAA2A012EF5D70AD0C40EA66EEECF70
:10015000F5FF0C0030D80900012EF7D700D0010EB2
:10016000016E0F0E1BD81AD8006A00EE08F0EE5090
:10017000002608D8012EFBD7006C005003D8040ECF
:100180000DD859D7056E0F0A06E00550040A03E0A2
:100190000550050A02E1050E01D8055004009EA88D
:1001A000FED7AD6E12000400ABB2FF009EAAFED7D0
:1001B000AE50046E12000400550EA76EAA0EA76E74
:0601C000A68200001200FF
:06020000FBEF0DF01200FF
:020206000000F6
:0802080000018B918B93200E85
:100210008C6F080E916F8DC08FF08EC090F08F1F85
:10022000901F120000018BB10FD00001BCB10CD0A7
:100230000001C36B0001010EC26F00019A0EC16F75
:10024000DBEC0AF000018B8100018BB30DD00001C3
:10025000BCB1A3D10001C06B00019A0EBF6FCFECFF
:100260000AF000018B831200915102E09107120005
:10027000080E916F8C5117E00001BCA986D10001D6
:100280008C07BBC028F0296A28BE29688D51282414
:100290008D6F8E5129208E6F030E8D27000E8E23B9
:1002A0000001BC9972D1200E1F6E206A8DC01AF019
:1002B0008EC01BF034EC0DF01AC08DF01BC08EF018
:1002C0001AC028F01BC029F0200E1F6E206A34ECE3
:1002D0000DF016C028F017C029F01750000AE8AE3C
:1002E00002D0293405D0100ED8802854000E29548D
:1002F00004E200018D2B000E8E2300018D518F1919
:1003000002E18E51901901E13BD18DC08FF08EC07A
:1003100090F0200E9D6F9C6F9B6F9A6F996F990E56
:10032000E66E000EE66E8DC0E6FF8EC0E6FFBFEC07
:1003300009F0E552E552E552E5520001390E866FAB
:10034000090E876F000E886FA8EC03F00001050E00
:10035000986F0001980E846F000E856F37EC03F0E4
:100360000001200E9D6F9C6F9B6F9A6F996F8DC0DF
:1003700028F08EC029F0030ED89028362936E806DA
:10038000FBE10A0E1F6E206A28C01AF029C01BF07C
:1003900034EC0DF01AC028F01BC029F0200E2826DE
:1003A000000E2922285000018D25946F29508E219E
:1003B000956F8DC028F08EC029F0030ED890283696
:1003C0002936E806FBE10A0E1F6E206A28C01AF0E3
:1003D00029C01BF034EC0DF016C028F017C029F02E
:1003E0001750000AE8AE02D0293405D0050ED88097
:1003F0002854000E295404E20001942B000E95238A
:10040000990EE66E000EE66E94C0E6FF95C0E6FF1C
:10041000BFEC09F0E552E552E552E5520001410E0C
:10042000866F090E876F000E886FA8EC03F000013D
:10043000050E986F0001980E846F000E856F37ECE3
:1004400003F00001200E9D6F9C6F9B6F9A6F996F58
:10045000110E8D25926F010E8E21936F990EE66E0F
:10046000000EE66E92C0E6FF93C0E6FFBFEC09F017
:10047000E552E552E552E5520001490E866F090E3C
:10048000876F000E886FA8EC03F00001050E986FCF
:100490000001980E846F000E856F37EC03F00001A9
:1004A000200E9D6F9C6F9B6F9A6F996F8DC028F087
:1004B0008EC029F0030ED89028362936E806FBE1D5
:1004C0000A0E1F6E206A28C01AF029C01BF034ECF7
:1004D0000DF01AC028F01BC029F0EC0E2826010EE2
:1004E0002922285000018D25966F29508E21976F63
:1004F0008DC028F08EC029F0030ED89028362936FA
:10050000E806FBE10A0E1F6E206A28C01AF029C017
:100510001BF034EC0DF016C028F017C029F017506E
:10052000000AE8AE02D0293405D0050ED880285440
:10053000000E295404E20001962B000E9723990E19
:10054000E66E000EE66E96C0E6FF97C0E6FFBFECD3
:1005500009F0E552E552E552E5520001510E866F71
:10056000090E876F000E886FA8EC03F00001050EDE
:10057000986F0001980E846F000E856F37EC03F0C2
:100580000001200E8C6F8D6B8E6B0001BCB105D00D
:0C05900000019A0EC46FE9EC0AF01200A2
:04059C0083C082F0A6
:1005A000000E0001796F7A6B776F786B8193AB6A7D
:1005B000900EAB6EAC6A240EAC6E83C0AFFF010C24
:1005C000120000018151020B43E0AC50020B40E0ED
:1005D0007DC0E9FF7EC0EAFFEF50AD6E7F077F511F
:1005E00034E17951771911E17A5178190EE177C028
:1005F00007F078C008F0A6EC08F0000E0001796F53
:100600007A6B776F786B819323D077C0E9FF78C0DE
:10061000EAFFEE52EECF7BF0EDCF7CF0030E7B25B0
:100620007D6F000E7C217E6F77C0E9FF78C0EAFF06
:10063000EFCF7FF077C007F078C008F0A6EC08F0A5
:100640007BC077F07CC078F003D07D2B000E7E233A
:10065000AB50040B03E1AB50020B08E0AB6A900E09
:10066000AB6EAC6A240EAC6E82C0AFFF120084C0C9
:10067000E9FF85C0EAFFEF50286E296A010E28269F
:10068000000E2922020E28240001006F43EC08F01E
:10069000F3CF7BF0F4CF7CF00001F350F41057E07F
:1006A0007751781119E17BC079F07CC07AF07BC07A
:1006B00077F07CC078F084C0E9FF85C0EAFFEFCF17
:1006C0007FF0010E77257D6F000E78217E6F020E80
:1006D0007D27000E7E231AD079C0E9FF7AC0EAFF99
:1006E000EE527BC0EEFF7CC0EDFF84C0E9FF85C009
:1006F000EAFFEF50E66E79C0E9FF7AC0EAFFE55203
:10070000E750EF6E7BC079F07CC07AF084C0E9FFDF
:1007100085C0EAFFEF500001B06FB16B030E00011E
:100720007B250001AE6F000E00017C210001AF6F40
:10073000010E000184250001AC6F000E000185212F
:100740000001AD6F8AEC05F000018183010C000C03
:1007500086C0F6FF87C0F7FF88C0F8FF0800F55095
:10076000286E296A010E2826000E2922020E28244E
:100770000001006F43EC08F0F3CF7BF0F4CF7CF086
:100780000001F350F41061E0775178111CE17BC057
:1007900079F07CC07AF07BC077F07CC078F086C0BE
:1007A000F6FF87C0F7FF88C0F8FF0800F5CF7FF09D
:1007B000010E77257D6F000E78217E6F020E7D275A
:1007C000000E7E231DD079C0E9FF7AC0EAFFEE5209
:1007D0007BC0EEFF7CC0EDFF86C0F6FF87C0F7FF51
:1007E00088C0F8FF0800F550E66E79C0E9FF7AC0CE
:1007F000EAFFE552E750EF6E7BC079F07CC07AF0FB
:1008000086C0F6FF87C0F7FF88C0F8FF0800F550E4
:100810000001B76FB86B030E00017B250001B56FB7
:10082000000E00017C210001B66F86C0B2F087C0C7
:10083000B3F088C0B4F00001B22B000EB323B42390
:1008400059EC06F000018183010C000C12009EAAF5
:0808500002D0AE501200000CB2
:08085800031B5B66031B5B4AF6
:10086000020D0A5B50494344454D20485043204502
:1008700078706C6F7265720A0D004D6963726F63F8
:1008800068697020546563686E6F6C6F6779204982
:100890006E632E0A0D0044656D6F206669726D7778
:1008A0006172652076312E30300A0D004E6F76650C
:1008B0006D62657220322C20323030340A0D000B0C
:1008C000526F737320466F736C65720A0D00691B5B
:1008D0005B363B316654656D706572617475726527
:1008E000202843656C73697573293A0A0D005465B5
:1008F0006D706572617475726520284661687265F5
:100900006E68656974293A0A0D0054656D706572E8
:10091000617475726520284B656C76696E293A0A98
:100920000D0054656D706572617475726520285292
:10093000616E6B696E65293A00071B5B363B323787
:1009400066071B5B373B323766071B5B383B32372A
:1009500066071B5B393B323766211B5B31313B310C
:1009600066504F5420566F6C746167653A200A0DCB
:1009700000504F542056616C75653A00081B5B317E
:10098000313B313466081B5B31323B3134663F1BEF
:100990005B31343B31664C4544733A20202044316E
:1009A00020202044322020204433202020443420A2
:1009B0002020443520202044362020204437202089
:1009C0002044380A0D005374617475733A2000078F
:1009D0001B5B31353B3966054F6E20202000054FEB
:1009E0006666202000131B5B31373B31664275740D
:1009F000746F6E205242303A2000081B5B31373B47
:100A00003133660B507265737365642020202000BB
:100A10000B4E6F74207072657373656400241B5BEA
:100A200032323B316650726573732027622720741F
:100A30006F20656E74657220626F6F74206D6F64D5
:100A4000652E00121B5B31393B316654696D653A86
:100A5000200007081B5B31393B3131663F1B5B3798
:100A60003B3166456E746572696E6720626F6F74A4
:100A7000206D6F64652077696C6C20666F726365AA
:100A8000207468652064656D6F206669726D77619A
:100A9000726520746F2073746F700A0D0053667551
:100AA0006E6374696F6E696E672E20416E79207077
:100AB000726F6772616D6D696E67206F70657261CC
:100AC00074696F6E20746865726520616674657202
:100AD000206D61790A0D0064657374726F792074FA
:100AE00068652064656D6F20636F64652E0A0D0A6A
:100AF0000D001F446F20796F752077616E7420742C
:100B00006F20656E74657220626F6F74206D6F6404
:030B1000653F003E
:0C0B14000001B051B11101E1C9D0040E84
:100B2000B05D000EB15911E2ACC0E9FFADC0EAFF03
:100B3000EF50AEC0E9FFAFC0EAFFEF6EAE2B000E84
:100B4000AF23AC2BAD23B007B1D0080EB05D000EC3
:100B5000B15922E2ACC0E9FFADC0EAFFEECF28F008
:100B6000EECF29F0EECF2AF0EFCF2BF0AEC0E9FFA9
:100B7000AFC0EAFF28C0EEFF29C0EEFF2AC0EEFF9B
:100B80002BC0EEFF040EAE27000EAF23040EAC27E1
:100B9000000EAD23040E88D0100EB05D000EB159CA
:100BA00032E2ACC0E9FFADC0EAFFEECF28F0EECFF5
:100BB00029F0EECF2AF0EECF2BF0EECF2CF0EECFD7
:100BC0002DF0EECF2EF0EFCF2FF0AEC0E9FFAFC08B
:100BD000EAFF28C0EEFF29C0EEFF2AC0EEFF2BC0BF
:100BE000EEFF2CC0EEFF2DC0EEFF2EC0EEFF2FC09B
:100BF000EEFF080EAE27000EAF23080EAC27000E46
:100C0000AD23080E51D0ACC0E9FFADC0EAFFEECF76
:100C100028F0EECF29F0EECF2AF0EECF2BF0EECF7A
:100C20002CF0EECF2DF0EECF2EF0EECF2FF0EECF5A
:100C300030F0EECF31F0EECF32F0EECF33F0EECF3A
:100C400034F0EECF35F0EECF36F0EFCF37F0AEC068
:100C5000E9FFAFC0EAFF28C0EEFF29C0EEFF2AC0BF
:100C6000EEFF2BC0EEFF2CC0EEFF2DC0EEFF2EC01E
:100C7000EEFF2FC0EEFF30C0EEFF31C0EEFF32C0FE
:100C8000EEFF33C0EEFF34C0EEFF35C0EEFF36C0DE
:100C9000EEFF37C0EEFF100EAE27000EAF23100E92
:100CA000AC27000EAD23100EB05F000EB15B32D743
:100CB00012000001B751B81101E188D0040EB75DF0
:100CC000000EB85915E2B2C0F6FFB3C0F7FFB4C0CA
:100CD000F8FF0800F550B5C0E9FFB6C0EAFFEF6EB7
:100CE000B52B000EB623B22BB323B423B7076CD0B9
:100CF000080EB75D000EB85929E2B2C0F6FFB3C0C6
:100D0000F7FFB4C0F8FF0900F5CF28F00900F5CFD0
:100D100029F00900F5CF2AF00800F5CF2BF0B5C077
:100D2000E9FFB6C0EAFF28C0EEFF29C0EEFF2AC0E7
:100D3000EEFF2BC0EEFF040EB527000EB623040E07
:100D4000B227000EB323B423040E3CD0B2C0F6FF8A
:100D5000B3C0F7FFB4C0F8FF0900F5CF28F00900D1
:100D6000F5CF29F00900F5CF2AF00900F5CF2BF0D7
:100D70000900F5CF2CF00900F5CF2DF00900F5CFD3
:100D80002EF00800F5CF2FF0B5C0E9FFB6C0EAFF9E
:100D900028C0EEFF29C0EEFF2AC0EEFF2BC0EEFFF9
:100DA0002CC0EEFF2DC0EEFF2EC0EEFF2FC0EEFFD9
:100DB000080EB527000EB623080EB227000EB32387
:0E0DC000B423080EB75F000EB85B73D71200A5
:020DCE00010E14
:100DD000C26EC16A830EC06E0001400E606F61C0BA
:100DE00063F062C064F0631F641F12009EAC49D1BF
:100DF0009E9C0001605108E060076151C324616F4F
:100E00006251C420626F120061C028F062C029F0F4
:100E1000060ED89029322832E804FBE128C061F0A0
:100E200029C062F000012850631902E1625164197F
:100E300001E121D161C063F062C064F00001850E60
:100E4000866F090E876F000E886FA8EC03F0000113
:100E5000200E766F756F746F736F726F720EE66E21
:100E6000000EE66E61C0E6FF62C0E6FFBFEC09F06F
:100E7000E552E552E552E5520001050E716F0001A1
:100E8000710E846F000E856F37EC03F000017C0E4D
:100E9000866F090E876F000E886FA8EC03F00001C3
:100EA000200E766F756F746F726F050E1A6E1B6A67
:100EB00061C01FF062C020F05AEC0DF018C065F060
:100EC00019C066F01F68030E206E18C01AF019C012
:100ED0001BF0D4EC0DF01AC065F01BC066F00001E9
:100EE000676B686B720EE66E000EE66E1AC0E6FF68
:100EF0001BC0E6FFBFEC09F0E552E552E552E552B2
:100F000000012E0E736F050E1A6E1B6A61C01FF072
:100F100062C020F05AEC0DF018C065F019C066F000
:100F20001F68030E206E18C01AF019C01BF0D4EC15
:100F30000DF016C065F017C066F000010A0E6603DA
:100F4000F3CF66F06503F3CF65F0F4506627676B67
:100F5000686BF3CF69F066C06AF067C06BF068C079
:100F60006CF01D68030E1E6E1F6A206AF3CF18F026
:100F700066C019F067C01AF068C01BF0B0EC0DF045
:100F800018C069F019C06AF01AC06BF01BC06CF091
:100F9000740EE66E000EE66E18C0E6FF19C0E6FF9E
:100FA000BFEC09F0E552E552E552E55265C069F043
:100FB00066C06AF067C06BF068C06CF01D68030E15
:100FC0001E6E1F6A206A65C018F066C019F067C0FF
:100FD0001AF068C01BF0B0EC0DF014C069F015C039
:100FE0006AF016C06BF017C06CF00A0E1D6E1E6A18
:100FF0001F6A206A14C018F015C019F016C01AF044
:1010000017C01BF078EC0DF014C069F015C06AF041
:1010100016C06BF017C06CF01D68030E1E6E1F6AC1
:10102000206A14C018F015C019F016C01AF017C0C5
:101030001BF0B0EC0DF018C069F019C06AF01AC0CE
:101040006BF01BC06CF0750EE66E000EE66E18C0FD
:10105000E6FF19C0E6FFBFEC09F0E552E552E552A4
:10106000E5520001050E716F0001710E846F000ED4
:10107000856F37EC03F00001400E606F616B626BAF
:061080001200C282120002
:0A10860000507E0810E3000E016E1A
:101090000A0E026E01C0E9FF02C0EAFFEF50056EC2
:1010A000E8507F0BFF0F066E055003E1F36AF46A08
:1010B000120005BE42D00650D880005408E201C09C
:1010C0000DF002C00EF074D80009E4E136D00650ED
:1010D000005C0EE101C0E9FF02C0EAFFEF8E010EE5
:1010E0000124286E000E022028C0F3FFF46E1200C7
:1010F000810E0024E66E01C0E9FF02C0EAFFE5525E
:10110000E750EF6E010E0124036E000E0220046E04
:101110000028296AE8500126295002220050065C66
:10112000E66E01C0E9FF02C0EAFFE552E750EF6E4C
:1011300003C0F3FF04C0F4FF120005507F0B286EBC
:10114000296AE850012629500222A4D707C0E9FFE6
:1011500008C0EAFFE906000EEA5AEF9E1200000EF0
:10116000096E0A0E0A6E0B68020E0C6E7F0ED88096
:101170000B54000E0C540EE209C0E9FF0AC0EAFF4E
:101180007F0EEF6E0926000E0A227F0E0B5E000E08
:101190000C5AECD709C0E9FF0AC0EAFF0BC0EFFF09
:1011A00009500B24E96E0A500C20EA6EEF6A120017
:1011B0000DC0E9FF0EC0EAFFEF5000010D240F6FD4
:1011C000000E0E20106FEF50116E0FC0E9FF10C01F
:1011D000EAFFEF50126EE85001E1000C1150800B55
:1011E00003E11250800B01E0000C11507F0B7F08CF
:1011F00001E1000C11501224136EE8507F081BE22D
:101200000DC0E9FF0EC0EAFF7F0EEF6E0D26000E47
:101210000E221250296A12500F26295010220D500A
:101220000F5C286E0E5010580DC0E9FF0EC0EAFF8B
:1012300028C0EFFF7F0C0DC0E9FF0EC0EAFF13C00E
:06124000EFFFEF50120069
:0A1246008C68956A12000001CF0EBB
:10125000866F090E876F000E886FA8EC03F08CA0D4
:1012600007D00001D70E866F090E876F000E06D0DB
:101270000001DE0E866F090E876F000E886FA8ECE6
:1012800003F08CA207D00001D70E866F090E876F7E
:10129000000E06D00001DE0E866F090E876F000E6D
:1012A000886FA8EC03F08CA407D00001D70E866FDE
:1012B000090E876F000E06D00001DE0E866F090E44
:1012C000876F000E886FA8EC03F08CA607D0000192
:1012D000D70E866F090E876F000E06D00001DE0E56
:1012E000866F090E876F000E886FA8EC03F08CA83C
:1012F00007D00001D70E866F090E876F000E06D04B
:101300000001DE0E866F090E876F000E886FA8EC55
:1013100003F08CAA07D00001D70E866F090E876FE5
:10132000000E06D00001DE0E866F090E876F000EDC
:10133000886FA8EC03F08CAC07D00001D70E866F45
:10134000090E876F000E06D00001DE0E866F090EB3
:10135000876F000E886FA8EC03F08CAE07D00001F9
:10136000D70E866F090E876F000E06D00001DE0EC5
:0E137000866F090E876F000E886FA8EF03F0DE
:02137E00D9CFC5
:10138000E6FFDACFE6FFFA0EE3CFD9FFFB0EE3CF9D
:10139000DAFFFD0EE35209E72D0EDE6EFC0EE31EB2
:1013A000E32AFD0ED8B4E306E31EE652E652E65207
:1013B000FD0EE124E76EFF0EE220E46EE652F70E2A
:1013C000E3CFE6FFF70EE3CFE6FF2FEC0AF0F90ECE
:1013D000E124E96EFF0EE220EA6E1FEC0AF00AE15A
:1013E0001CEC0AF009E11FEC0AF008E11CEC0AF021
:1013F00007E108D02AEC0AF025EC0AF02AEC0AF002
:1014000025EC0AF02AEC0AF0DE6AF90EE126FF0E5E
:10141000E222FF0EE3CFDAFFE552FF0EE3CFD9FF62
:10142000E552FC0EE124E96EFF0EE220EA6EEECFFB
:10143000F3FFEFCFF4FF1200EF380F0B1200EF5065
:101440000F0B02E1EE52D8841200EF380F0B300F71
:10145000DE6E1200EE500F0B300FDE6E1200FC0E2F
:10146000E3CFE9FFFD0EE3CFEAFF100EE66EEE6A72
:10147000EE6AEF6AD890FD0EE336FE0EE336ED36E7
:10148000ED36EF36FF0EE30609E050EC0AF0EE52BF
:1014900050EC0AF0EE5250EC0AF0EDD7E56E120077
:1014A000030EEF24E8B6EF6E300EEF24E8BEEF6EC9
:0214B000000C2E
:0E14B2000001BC6BBD6B8B868B889486948882
:1014C000C78E280EC66EC78CBEC0C8FF9E9612007F
:1014D0009EA664D09E960001BCA310D0BCB95ED07D
:1014E000BDA139D0BDA33CD0BDB503D0C5AC12D091
:1014F00015D0BDBB27D0C5AC4AD019D0BCA525D0CE
:10150000BCB94CD0BDA127D0BDA32AD0BDB508D051
:10151000C5BC04D0BAC0C9FFBD851200BD932CD094
:10152000BDB708D0C5BC03D0BBC0C9FF22D0BD9396
:10153000BD9522D0BDBB06D0C5AC29D0BD93BD950D
:10154000BD971AD0BC89BC911200BCA727D0BCB9EA
:1015500025D0BDB103D0C580BD811200BDB304D07C
:10156000B9C0C9FFBD831200BDB708D0C5BC03D048
:10157000C586BD871200BD93C5821200BDB905D0D6
:10158000C596C58AC588BD891200BDBB03D0C58478
:10159000BD8B1200C9CFBBF0BC89BC911200FE0EFE
:1015A0000001BF15B96FC0C0BAF0BD6BBC6BBC8188
:1015B000BC839E861200FE0E0001C115B96FC2C029
:1015C000BAF0C3C0BBF0BD6BBC6BBC81BC859E8652
:1015D0001200010E0001C411B96FBD6BBC6BBC8160
:0615E000BC879E8612008C
:0A15E6000F0ECD6E800ECF6ECE6AA0
:1015F0000001A16BA1C0A0F0A1C09EF012009EA0AE
:1016000065D09E90CF8E00019E2B00019E513B081D
:1016100012E200019E6B0001A02B0001A0513B08CB
:101620000AE20001A06B0001A12B0001A1511708E3
:1016300002E20001A16B00019E5100019F5D46E0A6
:101640009EC09FF00001530E866F0A0E876F000E3A
:10165000886FA8EC03F0A30EE66E000EE66E0001A4
:10166000A051E66EE66ABFEC09F0E552E552E5529C
:10167000E5520001A45105E1A3C0A4F00001300E21
:10168000A36F00013A0EA56FA60EE66E000EE66E81
:1016900000019E51E66EE66ABFEC09F0E552E552A4
:1016A000E552E5520001A75105E1A6C0A7F00001EF
:1016B000300EA66F0001A86B0001050EA26F00019D
:0E16C000A20E846F000E856F37EC03F012004F
:0216CE0081B0E9
:1016D00003D0FC6A02EF00F0AFEC08F0EAEC0DF08A
:1016E00000012B0E836FCEEC02F03CEC0CF023ECEF
:1016F00009F026EC09F0E7EC06F0E5EC0CF000014F
:101700007F0EBE6F59EC0AF004EC01F0F3EC0AF026
:10171000E1EC02F068EC0AF0F1EC0DF0000908E0F1
:10172000F6EC06F0FFEC0AF005EC0DF012EC01F01F
:1017300027EC04F00001CF6F0001CF51620A31E0C5
:101740005A0A2BE00F0A25E0010A1FE0030A19E0FC
:10175000010A13E0070A0DE0010A07E0030A01E0AD
:1017600023D08C7026EC09F01FD08C7226EC09F087
:101770001BD08C7426EC09F017D08C7626EC09F07F
:1017800013D08C7826EC09F00FD08C7A26EC09F077
:101790000BD08C7C26EC09F007D08C7E26EC09F06F
:0C17A00003D0D6EC0BF000D0B3D7120041
:0417AC000001580ED2
:1017B000866F080E876F000E886FA8EC03F000019B
:1017C0005C0E866F080E876F000E886FA8EC03F022
:1017D0000001580E866F080E876F000E886FA8EC08
:1017E00003F00001630E866F080E876F000E886F8E
:1017F000A8EC03F000015C0E866F0A0E876F000EE6
:10180000886FA8EC03F000019D0E866F0A0E876FAB
:10181000000E886FA8EC03F00001F20E866F0A0E2E
:10182000876F000E886FA8EC03F0E1EC02F068EC23
:101830000AF027EC04F00001D26F0001D25109E058
:10184000790A03E0200A01E005D0FC6A02EF00F00B
:1018500011D010D03CEC0CF0E7EC06F0F6EC06F002
:10186000E5EC0CF026EC09F004EC01F012EC01F0D0
:0818700002D000D0DAD712000B
:081878000001580E866F080EF6
:10188000876F000E886FA8EC03F000015C0E866F76
:10189000080E876F000E886FA8EC03F00001580E49
:1018A000866F080E876F000E886FA8EC03F00001AA
:1018B000630E866F080E876F000E886FA8EC03F02A
:1018C0000001CE0E866F080E876F000E886FA8ECA1
:1018D00003F00001590E866F090E876F000E886FA6
:1018E000A8EC03F000018E0E866F090E876F000EC4
:1018F000886FA8EC03F00001E50E866F090E876F74
:10190000000E886FA8EC03F000011D0E866F0A0E12
:10191000876F000E886FA8EC03F00001430E866FFE
:0C1920000A0E876F000E886FA8EF03F01E
:04192C00060EF66E3F
:10193000020EF76E000EF86E00010900F550CA6F36
:101940000900F550CB6F03E1CA6701D03DD0090013
:10195000F550C56F0900F550C66F0900F550C76F07
:1019600009000900F550E96E0900F550EA6E09001A
:1019700009000900F550C86F0900F550C96F09004A
:101980000900F6CFCCF0F7CFCDF0F8CFCEF0C5C040
:10199000F6FFC6C0F7FFC7C0F8FF0001C85302E159
:1019A000C95307E00900F550EE6EC807F8E2C90711
:1019B000F9D7CCC0F6FFCDC0F7FFCEC0F8FF0001CD
:0A19C000CA07000ECB5BBFD7120070
:0619CA000001FA0E866F19
:1019D000090E876F000E886FA8EC03F081A007D076
:1019E0000001100E866F0A0E876F000E06D00001F0
:1019F000030E866F0A0E876F000E886FA8EC03F047
:101A00008150010B0001D16F120081A013D00001A1
:101A1000D15125E10001FA0E866F090E876F000E85
:101A2000886FA8EC03F00001100E866F0A0E876F16
:101A3000000E12D00001D15112E00001FA0E866FA3
:101A4000090E876F000E886FA8EC03F00001030EEB
:101A5000866F0A0E876F000E886FA8EC03F0815026
:081A6000010B0001D16F12001F
:081A6800226A20AE3DEF0DF0F3
:101A70001F6C201EE86A2022221E1BAE45EF0DF0CF
:101A80001A6C1B1EE86A1B22221ED4EC0DF01BBE32
:101A900055EF0DF022AE000C1A6C1B1EE86A1B22DB
:101AA000166C171EE86A1722000C22BE4CEF0DF0D0
:101AB0002388FF0C1AC026F01A501F02F4CF19F029
:101AC000F3CF18F01B502002F4CF1BF0F3CF1AF025
:101AD0001F02F3501926F4501A22E86A1B222650DE
:101AE0002002F3501926F4501A22E86A1B22000C37
:101AF00018501D02F3CF14F0F4CF15F01E02F3506E
:101B00001526000EF420166E18501F02F3501626EC
:101B1000000EF420176E18502002F35017261950AB
:101B20001D02F3501526F4501622000E17221950EC
:101B30001E02F3501626F450172219501F02F350BC
:101B400017261A501D02F3501626F45017221A5069
:101B50001E02F35017261B501D02F35017261200C9
:101B6000176A166A156A146A200EE76ED89018363E
:101B700019361A361B3614361536163617361D50DA
:101B8000145C1E5015581F5016582050175809E362
:101B90001D50145E1E50155A1F50165A2050175AC9
:081BA000182AE72EE4D7120019
:081BA800176A166A100EE76EC1
:101BB000D8901A361B36163617361F50165C205032
:101BC000175805E31F50165E2050175A1A2AE72EA1
:041BD000F0D7120038
:0C1BD400470ED56EC70ED66ED58EF2946B
:101BE0001200F2A407D00001C80ED06FE850D6262C
:061BF000F294010C000C50
:0A1BF6001DEE00F02DEE00F0F86A7D
:0E1C0000239C96EC0CF067EC0BF0FDD7120065
:020000040030CA
:08000000FFF6EEFEFFFFBBFF5F
:00000001FF
